
D:\STM32\Program\1.11_Odchudzanie\um0427\FWLib\project\RIDE\STM3210E-EVAL\stm32f10x_nvic.o:     file format elf32-littlearm
D:\STM32\Program\1.11_Odchudzanie\um0427\FWLib\project\RIDE\STM3210E-EVAL\stm32f10x_nvic.o

Disassembly of section .text.NVIC_DeInit:

00000000 <NVIC_DeInit>:
NVIC_DeInit():
D:\STM32\Program\1.11_Odchudzanie\um0427\FWLib\library\src/stm32f10x_nvic.c:40
   0:	4b0b      	ldr	r3, [pc, #44]	(30 <NVIC_DeInit+0x30>)
   2:	f04f 31ff 	mov.w	r1, #4294967295	; 0xffffffff
D:\STM32\Program\1.11_Odchudzanie\um0427\FWLib\library\src/stm32f10x_nvic.c:41
   6:	f06f 4270 	mvn.w	r2, #4026531840	; 0xf0000000
D:\STM32\Program\1.11_Odchudzanie\um0427\FWLib\library\src/stm32f10x_nvic.c:40
   a:	f8c3 1080 	str.w	r1, [r3, #128]
D:\STM32\Program\1.11_Odchudzanie\um0427\FWLib\library\src/stm32f10x_nvic.c:41
   e:	f8c3 2084 	str.w	r2, [r3, #132]
D:\STM32\Program\1.11_Odchudzanie\um0427\FWLib\library\src/stm32f10x_nvic.c:42
  12:	f8c3 1180 	str.w	r1, [r3, #384]
D:\STM32\Program\1.11_Odchudzanie\um0427\FWLib\library\src/stm32f10x_nvic.c:43
  16:	f8c3 2184 	str.w	r2, [r3, #388]
  1a:	3101      	adds	r1, #1
D:\STM32\Program\1.11_Odchudzanie\um0427\FWLib\library\src/stm32f10x_nvic.c:47
  1c:	4a04      	ldr	r2, [pc, #16]	(30 <NVIC_DeInit+0x30>)
  1e:	008b      	lsls	r3, r1, #2
D:\STM32\Program\1.11_Odchudzanie\um0427\FWLib\library\src/stm32f10x_nvic.c:45
  20:	3101      	adds	r1, #1
D:\STM32\Program\1.11_Odchudzanie\um0427\FWLib\library\src/stm32f10x_nvic.c:47
  22:	189a      	adds	r2, r3, r2
  24:	2300      	movs	r3, #0
D:\STM32\Program\1.11_Odchudzanie\um0427\FWLib\library\src/stm32f10x_nvic.c:45
  26:	290f      	cmp	r1, #15
D:\STM32\Program\1.11_Odchudzanie\um0427\FWLib\library\src/stm32f10x_nvic.c:47
  28:	f8c2 3300 	str.w	r3, [r2, #768]
D:\STM32\Program\1.11_Odchudzanie\um0427\FWLib\library\src/stm32f10x_nvic.c:45
  2c:	d1f6      	bne.n	1c <NVIC_DeInit+0x1c>
D:\STM32\Program\1.11_Odchudzanie\um0427\FWLib\library\src/stm32f10x_nvic.c:49
  2e:	4770      	bx	lr
  30:	e000e100 	.word	0xe000e100
Disassembly of section .text.NVIC_SCBDeInit:

00000000 <NVIC_SCBDeInit>:
NVIC_SCBDeInit():
D:\STM32\Program\1.11_Odchudzanie\um0427\FWLib\library\src/stm32f10x_nvic.c:63
   0:	4a09      	ldr	r2, [pc, #36]	(28 <NVIC_SCBDeInit+0x28>)
   2:	f04f 6320 	mov.w	r3, #167772160	; 0xa000000
D:\STM32\Program\1.11_Odchudzanie\um0427\FWLib\library\src/stm32f10x_nvic.c:65
   6:	4909      	ldr	r1, [pc, #36]	(2c <NVIC_SCBDeInit+0x2c>)
D:\STM32\Program\1.11_Odchudzanie\um0427\FWLib\library\src/stm32f10x_nvic.c:63
   8:	6053      	str	r3, [r2, #4]
D:\STM32\Program\1.11_Odchudzanie\um0427\FWLib\library\src/stm32f10x_nvic.c:64
   a:	f103 4376 	add.w	r3, r3, #4127195136	; 0xf6000000
   e:	6093      	str	r3, [r2, #8]
D:\STM32\Program\1.11_Odchudzanie\um0427\FWLib\library\src/stm32f10x_nvic.c:65
  10:	60d1      	str	r1, [r2, #12]
D:\STM32\Program\1.11_Odchudzanie\um0427\FWLib\library\src/stm32f10x_nvic.c:66
  12:	6113      	str	r3, [r2, #16]
D:\STM32\Program\1.11_Odchudzanie\um0427\FWLib\library\src/stm32f10x_nvic.c:67
  14:	6153      	str	r3, [r2, #20]
D:\STM32\Program\1.11_Odchudzanie\um0427\FWLib\library\src/stm32f10x_nvic.c:70
  16:	6193      	str	r3, [r2, #24]
  18:	61d3      	str	r3, [r2, #28]
  1a:	6213      	str	r3, [r2, #32]
D:\STM32\Program\1.11_Odchudzanie\um0427\FWLib\library\src/stm32f10x_nvic.c:72
  1c:	6253      	str	r3, [r2, #36]
D:\STM32\Program\1.11_Odchudzanie\um0427\FWLib\library\src/stm32f10x_nvic.c:73
  1e:	3b01      	subs	r3, #1
  20:	6293      	str	r3, [r2, #40]
D:\STM32\Program\1.11_Odchudzanie\um0427\FWLib\library\src/stm32f10x_nvic.c:74
  22:	62d3      	str	r3, [r2, #44]
D:\STM32\Program\1.11_Odchudzanie\um0427\FWLib\library\src/stm32f10x_nvic.c:75
  24:	6313      	str	r3, [r2, #48]
D:\STM32\Program\1.11_Odchudzanie\um0427\FWLib\library\src/stm32f10x_nvic.c:76
  26:	4770      	bx	lr
  28:	e000ed00 	.word	0xe000ed00
  2c:	05fa0000 	.word	0x05fa0000
Disassembly of section .text.NVIC_PriorityGroupConfig:

00000000 <NVIC_PriorityGroupConfig>:
NVIC_PriorityGroupConfig():
D:\STM32\Program\1.11_Odchudzanie\um0427\FWLib\library\src/stm32f10x_nvic.c:103
   0:	f040 60be 	orr.w	r0, r0, #99614720	; 0x5f00000
   4:	4b02      	ldr	r3, [pc, #8]	(10 <NVIC_PriorityGroupConfig+0x10>)
   6:	f440 2020 	orr.w	r0, r0, #655360	; 0xa0000
   a:	60d8      	str	r0, [r3, #12]
D:\STM32\Program\1.11_Odchudzanie\um0427\FWLib\library\src/stm32f10x_nvic.c:104
   c:	4770      	bx	lr
   e:	46c0      	nop			(mov r8, r8)
  10:	e000ed00 	.word	0xe000ed00
Disassembly of section .text.NVIC_Init:

00000000 <NVIC_Init>:
NVIC_Init():
D:\STM32\Program\1.11_Odchudzanie\um0427\FWLib\library\src/stm32f10x_nvic.c:117
   0:	b510      	push	{r4, lr}
D:\STM32\Program\1.11_Odchudzanie\um0427\FWLib\library\src/stm32f10x_nvic.c:127
   2:	78c3      	ldrb	r3, [r0, #3]
   4:	f890 e000 	ldrb.w	lr, [r0]
   8:	b353      	cbz	r3, 60 <NVIC_Init+0x60>
D:\STM32\Program\1.11_Odchudzanie\um0427\FWLib\library\src/stm32f10x_nvic.c:130
   a:	4b1b      	ldr	r3, [pc, #108]	(78 <NVIC_Init+0x78>)
D:\STM32\Program\1.11_Odchudzanie\um0427\FWLib\library\src/stm32f10x_nvic.c:134
   c:	7841      	ldrb	r1, [r0, #1]
D:\STM32\Program\1.11_Odchudzanie\um0427\FWLib\library\src/stm32f10x_nvic.c:130
   e:	68da      	ldr	r2, [r3, #12]
D:\STM32\Program\1.11_Odchudzanie\um0427\FWLib\library\src/stm32f10x_nvic.c:140
  10:	4c1a      	ldr	r4, [pc, #104]	(7c <NVIC_Init+0x7c>)
D:\STM32\Program\1.11_Odchudzanie\um0427\FWLib\library\src/stm32f10x_nvic.c:130
  12:	43d2      	mvns	r2, r2
  14:	f3c2 2202 	ubfx	r2, r2, #8, #3
D:\STM32\Program\1.11_Odchudzanie\um0427\FWLib\library\src/stm32f10x_nvic.c:134
  18:	f1c2 0304 	rsb	r3, r2, #4	; 0x4
  1c:	4099      	lsls	r1, r3
D:\STM32\Program\1.11_Odchudzanie\um0427\FWLib\library\src/stm32f10x_nvic.c:135
  1e:	230f      	movs	r3, #15
  20:	40d3      	lsrs	r3, r2
  22:	7882      	ldrb	r2, [r0, #2]
D:\STM32\Program\1.11_Odchudzanie\um0427\FWLib\library\src/stm32f10x_nvic.c:138
  24:	f00e 0003 	and.w	r0, lr, #3	; 0x3
D:\STM32\Program\1.11_Odchudzanie\um0427\FWLib\library\src/stm32f10x_nvic.c:135
  28:	4013      	ands	r3, r2
  2a:	430b      	orrs	r3, r1
D:\STM32\Program\1.11_Odchudzanie\um0427\FWLib\library\src/stm32f10x_nvic.c:140
  2c:	f00e 02fc 	and.w	r2, lr, #252	; 0xfc
  30:	1914      	adds	r4, r2, r4
D:\STM32\Program\1.11_Odchudzanie\um0427\FWLib\library\src/stm32f10x_nvic.c:138
  32:	00c0      	lsls	r0, r0, #3
D:\STM32\Program\1.11_Odchudzanie\um0427\FWLib\library\src/stm32f10x_nvic.c:137
  34:	011b      	lsls	r3, r3, #4
D:\STM32\Program\1.11_Odchudzanie\um0427\FWLib\library\src/stm32f10x_nvic.c:141
  36:	22ff      	movs	r2, #255
  38:	4082      	lsls	r2, r0
D:\STM32\Program\1.11_Odchudzanie\um0427\FWLib\library\src/stm32f10x_nvic.c:138
  3a:	4083      	lsls	r3, r0
D:\STM32\Program\1.11_Odchudzanie\um0427\FWLib\library\src/stm32f10x_nvic.c:140
  3c:	f8d4 1300 	ldr.w	r1, [r4, #768]
D:\STM32\Program\1.11_Odchudzanie\um0427\FWLib\library\src/stm32f10x_nvic.c:144
  40:	4013      	ands	r3, r2
D:\STM32\Program\1.11_Odchudzanie\um0427\FWLib\library\src/stm32f10x_nvic.c:142
  42:	ea21 0102 	bic.w	r1, r1, r2
D:\STM32\Program\1.11_Odchudzanie\um0427\FWLib\library\src/stm32f10x_nvic.c:144
  46:	430b      	orrs	r3, r1
D:\STM32\Program\1.11_Odchudzanie\um0427\FWLib\library\src/stm32f10x_nvic.c:146
  48:	f8c4 3300 	str.w	r3, [r4, #768]
D:\STM32\Program\1.11_Odchudzanie\um0427\FWLib\library\src/stm32f10x_nvic.c:149
  4c:	f00e 021f 	and.w	r2, lr, #31	; 0x1f
  50:	2301      	movs	r3, #1
  52:	4093      	lsls	r3, r2
  54:	4a09      	ldr	r2, [pc, #36]	(7c <NVIC_Init+0x7c>)
  56:	ea4f 115e 	mov.w	r1, lr, lsr #5
  5a:	f842 3021 	str.w	r3, [r2, r1, lsl #2]
  5e:	e00a      	b.n	76 <NVIC_Init+0x76>
D:\STM32\Program\1.11_Odchudzanie\um0427\FWLib\library\src/stm32f10x_nvic.c:155
  60:	f00e 031f 	and.w	r3, lr, #31	; 0x1f
  64:	2201      	movs	r2, #1
  66:	409a      	lsls	r2, r3
  68:	ea4f 115e 	mov.w	r1, lr, lsr #5
  6c:	4b03      	ldr	r3, [pc, #12]	(7c <NVIC_Init+0x7c>)
  6e:	0089      	lsls	r1, r1, #2
  70:	18cb      	adds	r3, r1, r3
  72:	f8c3 2080 	str.w	r2, [r3, #128]
D:\STM32\Program\1.11_Odchudzanie\um0427\FWLib\library\src/stm32f10x_nvic.c:158
  76:	bd10      	pop	{r4, pc}
  78:	e000ed00 	.word	0xe000ed00
  7c:	e000e100 	.word	0xe000e100
Disassembly of section .text.NVIC_StructInit:

00000000 <NVIC_StructInit>:
NVIC_StructInit():
D:\STM32\Program\1.11_Odchudzanie\um0427\FWLib\library\src/stm32f10x_nvic.c:171
   0:	2300      	movs	r3, #0
   2:	7003      	strb	r3, [r0, #0]
D:\STM32\Program\1.11_Odchudzanie\um0427\FWLib\library\src/stm32f10x_nvic.c:172
   4:	7043      	strb	r3, [r0, #1]
D:\STM32\Program\1.11_Odchudzanie\um0427\FWLib\library\src/stm32f10x_nvic.c:173
   6:	7083      	strb	r3, [r0, #2]
D:\STM32\Program\1.11_Odchudzanie\um0427\FWLib\library\src/stm32f10x_nvic.c:174
   8:	70c3      	strb	r3, [r0, #3]
D:\STM32\Program\1.11_Odchudzanie\um0427\FWLib\library\src/stm32f10x_nvic.c:175
   a:	4770      	bx	lr
Disassembly of section .text.NVIC_GetCurrentPendingIRQChannel:

00000000 <NVIC_GetCurrentPendingIRQChannel>:
NVIC_GetCurrentPendingIRQChannel():
D:\STM32\Program\1.11_Odchudzanie\um0427\FWLib\library\src/stm32f10x_nvic.c:263
   0:	4b02      	ldr	r3, [pc, #8]	(c <NVIC_GetCurrentPendingIRQChannel+0xc>)
   2:	6858      	ldr	r0, [r3, #4]
D:\STM32\Program\1.11_Odchudzanie\um0427\FWLib\library\src/stm32f10x_nvic.c:264
   4:	f3c0 3009 	ubfx	r0, r0, #12, #10
   8:	4770      	bx	lr
   a:	46c0      	nop			(mov r8, r8)
   c:	e000ed00 	.word	0xe000ed00
Disassembly of section .text.NVIC_GetIRQChannelPendingBitStatus:

00000000 <NVIC_GetIRQChannelPendingBitStatus>:
NVIC_GetIRQChannelPendingBitStatus():
D:\STM32\Program\1.11_Odchudzanie\um0427\FWLib\library\src/stm32f10x_nvic.c:282
   0:	f000 031f 	and.w	r3, r0, #31	; 0x1f
   4:	2201      	movs	r2, #1
   6:	409a      	lsls	r2, r3
D:\STM32\Program\1.11_Odchudzanie\um0427\FWLib\library\src/stm32f10x_nvic.c:284
   8:	0940      	lsrs	r0, r0, #5
   a:	4b05      	ldr	r3, [pc, #20]	(20 <NVIC_GetIRQChannelPendingBitStatus+0x20>)
   c:	0080      	lsls	r0, r0, #2
   e:	18c3      	adds	r3, r0, r3
  10:	f8d3 0100 	ldr.w	r0, [r3, #256]
  14:	4010      	ands	r0, r2
D:\STM32\Program\1.11_Odchudzanie\um0427\FWLib\library\src/stm32f10x_nvic.c:293
  16:	4290      	cmp	r0, r2
  18:	bf14      	ite	ne
  1a:	2000      	movne	r0, #0
  1c:	2001      	moveq	r0, #1
  1e:	4770      	bx	lr
  20:	e000e100 	.word	0xe000e100
Disassembly of section .text.NVIC_SetIRQChannelPendingBit:

00000000 <NVIC_SetIRQChannelPendingBit>:
NVIC_SetIRQChannelPendingBit():
D:\STM32\Program\1.11_Odchudzanie\um0427\FWLib\library\src/stm32f10x_nvic.c:307
   0:	4b01      	ldr	r3, [pc, #4]	(8 <NVIC_SetIRQChannelPendingBit+0x8>)
   2:	6018      	str	r0, [r3, #0]
D:\STM32\Program\1.11_Odchudzanie\um0427\FWLib\library\src/stm32f10x_nvic.c:308
   4:	4770      	bx	lr
   6:	46c0      	nop			(mov r8, r8)
   8:	e000ef00 	.word	0xe000ef00
Disassembly of section .text.NVIC_ClearIRQChannelPendingBit:

00000000 <NVIC_ClearIRQChannelPendingBit>:
NVIC_ClearIRQChannelPendingBit():
D:\STM32\Program\1.11_Odchudzanie\um0427\FWLib\library\src/stm32f10x_nvic.c:322
   0:	0941      	lsrs	r1, r0, #5
   2:	2201      	movs	r2, #1
   4:	f000 001f 	and.w	r0, r0, #31	; 0x1f
   8:	4082      	lsls	r2, r0
   a:	4b03      	ldr	r3, [pc, #12]	(18 <NVIC_ClearIRQChannelPendingBit+0x18>)
   c:	0089      	lsls	r1, r1, #2
   e:	18cb      	adds	r3, r1, r3
  10:	f8c3 2180 	str.w	r2, [r3, #384]
D:\STM32\Program\1.11_Odchudzanie\um0427\FWLib\library\src/stm32f10x_nvic.c:323
  14:	4770      	bx	lr
  16:	46c0      	nop			(mov r8, r8)
  18:	e000e100 	.word	0xe000e100
Disassembly of section .text.NVIC_GetCurrentActiveHandler:

00000000 <NVIC_GetCurrentActiveHandler>:
NVIC_GetCurrentActiveHandler():
D:\STM32\Program\1.11_Odchudzanie\um0427\FWLib\library\src/stm32f10x_nvic.c:335
   0:	4b02      	ldr	r3, [pc, #8]	(c <NVIC_GetCurrentActiveHandler+0xc>)
   2:	6858      	ldr	r0, [r3, #4]
D:\STM32\Program\1.11_Odchudzanie\um0427\FWLib\library\src/stm32f10x_nvic.c:336
   4:	0580      	lsls	r0, r0, #22
   6:	0d80      	lsrs	r0, r0, #22
   8:	4770      	bx	lr
   a:	46c0      	nop			(mov r8, r8)
   c:	e000ed00 	.word	0xe000ed00
Disassembly of section .text.NVIC_GetIRQChannelActiveBitStatus:

00000000 <NVIC_GetIRQChannelActiveBitStatus>:
NVIC_GetIRQChannelActiveBitStatus():
D:\STM32\Program\1.11_Odchudzanie\um0427\FWLib\library\src/stm32f10x_nvic.c:354
   0:	f000 031f 	and.w	r3, r0, #31	; 0x1f
   4:	2201      	movs	r2, #1
   6:	409a      	lsls	r2, r3
D:\STM32\Program\1.11_Odchudzanie\um0427\FWLib\library\src/stm32f10x_nvic.c:356
   8:	0940      	lsrs	r0, r0, #5
   a:	4b05      	ldr	r3, [pc, #20]	(20 <NVIC_GetIRQChannelActiveBitStatus+0x20>)
   c:	0080      	lsls	r0, r0, #2
   e:	18c3      	adds	r3, r0, r3
  10:	f8d3 0200 	ldr.w	r0, [r3, #512]
  14:	4010      	ands	r0, r2
D:\STM32\Program\1.11_Odchudzanie\um0427\FWLib\library\src/stm32f10x_nvic.c:365
  16:	4290      	cmp	r0, r2
  18:	bf14      	ite	ne
  1a:	2000      	movne	r0, #0
  1c:	2001      	moveq	r0, #1
  1e:	4770      	bx	lr
  20:	e000e100 	.word	0xe000e100
Disassembly of section .text.NVIC_GetCPUID:

00000000 <NVIC_GetCPUID>:
NVIC_GetCPUID():
D:\STM32\Program\1.11_Odchudzanie\um0427\FWLib\library\src/stm32f10x_nvic.c:377
   0:	4b01      	ldr	r3, [pc, #4]	(8 <NVIC_GetCPUID+0x8>)
   2:	6818      	ldr	r0, [r3, #0]
D:\STM32\Program\1.11_Odchudzanie\um0427\FWLib\library\src/stm32f10x_nvic.c:378
   4:	4770      	bx	lr
   6:	46c0      	nop			(mov r8, r8)
   8:	e000ed00 	.word	0xe000ed00
Disassembly of section .text.NVIC_SetVectorTable:

00000000 <NVIC_SetVectorTable>:
NVIC_SetVectorTable():
D:\STM32\Program\1.11_Odchudzanie\um0427\FWLib\library\src/stm32f10x_nvic.c:399
   0:	f021 4160 	bic.w	r1, r1, #3758096384	; 0xe0000000
   4:	f021 017f 	bic.w	r1, r1, #127	; 0x7f
   8:	4b01      	ldr	r3, [pc, #4]	(10 <NVIC_SetVectorTable+0x10>)
   a:	4301      	orrs	r1, r0
   c:	6099      	str	r1, [r3, #8]
D:\STM32\Program\1.11_Odchudzanie\um0427\FWLib\library\src/stm32f10x_nvic.c:400
   e:	4770      	bx	lr
  10:	e000ed00 	.word	0xe000ed00
Disassembly of section .text.NVIC_GenerateSystemReset:

00000000 <NVIC_GenerateSystemReset>:
NVIC_GenerateSystemReset():
D:\STM32\Program\1.11_Odchudzanie\um0427\FWLib\library\src/stm32f10x_nvic.c:411
   0:	4a01      	ldr	r2, [pc, #4]	(8 <NVIC_GenerateSystemReset+0x8>)
   2:	4b02      	ldr	r3, [pc, #8]	(c <NVIC_GenerateSystemReset+0xc>)
   4:	60da      	str	r2, [r3, #12]
D:\STM32\Program\1.11_Odchudzanie\um0427\FWLib\library\src/stm32f10x_nvic.c:412
   6:	4770      	bx	lr
   8:	05fa0004 	.word	0x05fa0004
   c:	e000ed00 	.word	0xe000ed00
Disassembly of section .text.NVIC_GenerateCoreReset:

00000000 <NVIC_GenerateCoreReset>:
NVIC_GenerateCoreReset():
D:\STM32\Program\1.11_Odchudzanie\um0427\FWLib\library\src/stm32f10x_nvic.c:423
   0:	4a01      	ldr	r2, [pc, #4]	(8 <NVIC_GenerateCoreReset+0x8>)
   2:	4b02      	ldr	r3, [pc, #8]	(c <NVIC_GenerateCoreReset+0xc>)
   4:	60da      	str	r2, [r3, #12]
D:\STM32\Program\1.11_Odchudzanie\um0427\FWLib\library\src/stm32f10x_nvic.c:424
   6:	4770      	bx	lr
   8:	05fa0001 	.word	0x05fa0001
   c:	e000ed00 	.word	0xe000ed00
Disassembly of section .text.NVIC_SystemLPConfig:

00000000 <NVIC_SystemLPConfig>:
NVIC_SystemLPConfig():
D:\STM32\Program\1.11_Odchudzanie\um0427\FWLib\library\src/stm32f10x_nvic.c:446
   0:	b121      	cbz	r1, c <NVIC_SystemLPConfig+0xc>
D:\STM32\Program\1.11_Odchudzanie\um0427\FWLib\library\src/stm32f10x_nvic.c:448
   2:	4a05      	ldr	r2, [pc, #20]	(18 <NVIC_SystemLPConfig+0x18>)
   4:	6913      	ldr	r3, [r2, #16]
   6:	ea40 0303 	orr.w	r3, r0, r3
   a:	e003      	b.n	14 <NVIC_SystemLPConfig+0x14>
D:\STM32\Program\1.11_Odchudzanie\um0427\FWLib\library\src/stm32f10x_nvic.c:452
   c:	4a02      	ldr	r2, [pc, #8]	(18 <NVIC_SystemLPConfig+0x18>)
   e:	6913      	ldr	r3, [r2, #16]
  10:	ea23 0300 	bic.w	r3, r3, r0
  14:	6113      	str	r3, [r2, #16]
D:\STM32\Program\1.11_Odchudzanie\um0427\FWLib\library\src/stm32f10x_nvic.c:454
  16:	4770      	bx	lr
  18:	e000ed00 	.word	0xe000ed00
Disassembly of section .text.NVIC_SystemHandlerConfig:

00000000 <NVIC_SystemHandlerConfig>:
NVIC_SystemHandlerConfig():
D:\STM32\Program\1.11_Odchudzanie\um0427\FWLib\library\src/stm32f10x_nvic.c:478
   0:	f000 001f 	and.w	r0, r0, #31	; 0x1f
   4:	2301      	movs	r3, #1
   6:	fa13 f000 	lsls.w	r0, r3, r0
D:\STM32\Program\1.11_Odchudzanie\um0427\FWLib\library\src/stm32f10x_nvic.c:480
   a:	b121      	cbz	r1, 16 <NVIC_SystemHandlerConfig+0x16>
D:\STM32\Program\1.11_Odchudzanie\um0427\FWLib\library\src/stm32f10x_nvic.c:482
   c:	4a05      	ldr	r2, [pc, #20]	(24 <NVIC_SystemHandlerConfig+0x24>)
   e:	6a53      	ldr	r3, [r2, #36]
  10:	ea40 0303 	orr.w	r3, r0, r3
  14:	e003      	b.n	1e <NVIC_SystemHandlerConfig+0x1e>
D:\STM32\Program\1.11_Odchudzanie\um0427\FWLib\library\src/stm32f10x_nvic.c:486
  16:	4a03      	ldr	r2, [pc, #12]	(24 <NVIC_SystemHandlerConfig+0x24>)
  18:	6a53      	ldr	r3, [r2, #36]
  1a:	ea23 0300 	bic.w	r3, r3, r0
  1e:	6253      	str	r3, [r2, #36]
D:\STM32\Program\1.11_Odchudzanie\um0427\FWLib\library\src/stm32f10x_nvic.c:488
  20:	4770      	bx	lr
  22:	46c0      	nop			(mov r8, r8)
  24:	e000ed00 	.word	0xe000ed00
Disassembly of section .text.NVIC_SystemHandlerPriorityConfig:

00000000 <NVIC_SystemHandlerPriorityConfig>:
NVIC_SystemHandlerPriorityConfig():
D:\STM32\Program\1.11_Odchudzanie\um0427\FWLib\library\src/stm32f10x_nvic.c:512
   0:	b530      	push	{r4, r5, lr}
D:\STM32\Program\1.11_Odchudzanie\um0427\FWLib\library\src/stm32f10x_nvic.c:521
   2:	4d0f      	ldr	r5, [pc, #60]	(40 <NVIC_SystemHandlerPriorityConfig+0x40>)
   4:	68eb      	ldr	r3, [r5, #12]
   6:	43db      	mvns	r3, r3
   8:	f3c3 2302 	ubfx	r3, r3, #8, #3
D:\STM32\Program\1.11_Odchudzanie\um0427\FWLib\library\src/stm32f10x_nvic.c:525
   c:	f1c3 0404 	rsb	r4, r3, #4	; 0x4
  10:	40a1      	lsls	r1, r4
D:\STM32\Program\1.11_Odchudzanie\um0427\FWLib\library\src/stm32f10x_nvic.c:526
  12:	24ff      	movs	r4, #255
  14:	fa34 f303 	lsrs.w	r3, r4, r3
  18:	401a      	ands	r2, r3
D:\STM32\Program\1.11_Odchudzanie\um0427\FWLib\library\src/stm32f10x_nvic.c:530
  1a:	f3c0 1381 	ubfx	r3, r0, #6, #2
D:\STM32\Program\1.11_Odchudzanie\um0427\FWLib\library\src/stm32f10x_nvic.c:532
  1e:	f3c0 2001 	ubfx	r0, r0, #8, #2
  22:	00c0      	lsls	r0, r0, #3
D:\STM32\Program\1.11_Odchudzanie\um0427\FWLib\library\src/stm32f10x_nvic.c:535
  24:	4084      	lsls	r4, r0
D:\STM32\Program\1.11_Odchudzanie\um0427\FWLib\library\src/stm32f10x_nvic.c:526
  26:	430a      	orrs	r2, r1
D:\STM32\Program\1.11_Odchudzanie\um0427\FWLib\library\src/stm32f10x_nvic.c:528
  28:	0112      	lsls	r2, r2, #4
D:\STM32\Program\1.11_Odchudzanie\um0427\FWLib\library\src/stm32f10x_nvic.c:536
  2a:	4082      	lsls	r2, r0
D:\STM32\Program\1.11_Odchudzanie\um0427\FWLib\library\src/stm32f10x_nvic.c:535
  2c:	eb05 0583 	add.w	r5, r5, r3, lsl #2
  30:	69ab      	ldr	r3, [r5, #24]
  32:	ea23 0304 	bic.w	r3, r3, r4
  36:	61ab      	str	r3, [r5, #24]
D:\STM32\Program\1.11_Odchudzanie\um0427\FWLib\library\src/stm32f10x_nvic.c:536
  38:	69ab      	ldr	r3, [r5, #24]
  3a:	431a      	orrs	r2, r3
  3c:	61aa      	str	r2, [r5, #24]
D:\STM32\Program\1.11_Odchudzanie\um0427\FWLib\library\src/stm32f10x_nvic.c:537
  3e:	bd30      	pop	{r4, r5, pc}
  40:	e000ed00 	.word	0xe000ed00
Disassembly of section .text.NVIC_GetSystemHandlerPendingBitStatus:

00000000 <NVIC_GetSystemHandlerPendingBitStatus>:
NVIC_GetSystemHandlerPendingBitStatus():
D:\STM32\Program\1.11_Odchudzanie\um0427\FWLib\library\src/stm32f10x_nvic.c:563
   0:	f3c0 2083 	ubfx	r0, r0, #10, #4
   4:	2301      	movs	r3, #1
   6:	4083      	lsls	r3, r0
D:\STM32\Program\1.11_Odchudzanie\um0427\FWLib\library\src/stm32f10x_nvic.c:565
   8:	4a04      	ldr	r2, [pc, #16]	(1c <NVIC_GetSystemHandlerPendingBitStatus+0x1c>)
   a:	6a50      	ldr	r0, [r2, #36]
   c:	ea03 0000 	and.w	r0, r3, r0
D:\STM32\Program\1.11_Odchudzanie\um0427\FWLib\library\src/stm32f10x_nvic.c:576
  10:	4298      	cmp	r0, r3
  12:	bf14      	ite	ne
  14:	2000      	movne	r0, #0
  16:	2001      	moveq	r0, #1
  18:	4770      	bx	lr
  1a:	46c0      	nop			(mov r8, r8)
  1c:	e000ed00 	.word	0xe000ed00
Disassembly of section .text.NVIC_SetSystemHandlerPendingBit:

00000000 <NVIC_SetSystemHandlerPendingBit>:
NVIC_SetSystemHandlerPendingBit():
D:\STM32\Program\1.11_Odchudzanie\um0427\FWLib\library\src/stm32f10x_nvic.c:600
   0:	f000 001f 	and.w	r0, r0, #31	; 0x1f
   4:	2301      	movs	r3, #1
   6:	4083      	lsls	r3, r0
   8:	4a02      	ldr	r2, [pc, #8]	(14 <NVIC_SetSystemHandlerPendingBit+0x14>)
   a:	6851      	ldr	r1, [r2, #4]
   c:	430b      	orrs	r3, r1
   e:	6053      	str	r3, [r2, #4]
D:\STM32\Program\1.11_Odchudzanie\um0427\FWLib\library\src/stm32f10x_nvic.c:601
  10:	4770      	bx	lr
  12:	46c0      	nop			(mov r8, r8)
  14:	e000ed00 	.word	0xe000ed00
Disassembly of section .text.NVIC_ClearSystemHandlerPendingBit:

00000000 <NVIC_ClearSystemHandlerPendingBit>:
NVIC_ClearSystemHandlerPendingBit():
D:\STM32\Program\1.11_Odchudzanie\um0427\FWLib\library\src/stm32f10x_nvic.c:624
   0:	f000 001f 	and.w	r0, r0, #31	; 0x1f
   4:	3801      	subs	r0, #1
   6:	2301      	movs	r3, #1
   8:	4083      	lsls	r3, r0
   a:	4a02      	ldr	r2, [pc, #8]	(14 <NVIC_ClearSystemHandlerPendingBit+0x14>)
   c:	6851      	ldr	r1, [r2, #4]
   e:	430b      	orrs	r3, r1
  10:	6053      	str	r3, [r2, #4]
D:\STM32\Program\1.11_Odchudzanie\um0427\FWLib\library\src/stm32f10x_nvic.c:625
  12:	4770      	bx	lr
  14:	e000ed00 	.word	0xe000ed00
Disassembly of section .text.NVIC_GetSystemHandlerActiveBitStatus:

00000000 <NVIC_GetSystemHandlerActiveBitStatus>:
NVIC_GetSystemHandlerActiveBitStatus():
D:\STM32\Program\1.11_Odchudzanie\um0427\FWLib\library\src/stm32f10x_nvic.c:655
   0:	f3c0 3083 	ubfx	r0, r0, #14, #4
   4:	2301      	movs	r3, #1
   6:	4083      	lsls	r3, r0
D:\STM32\Program\1.11_Odchudzanie\um0427\FWLib\library\src/stm32f10x_nvic.c:657
   8:	4a04      	ldr	r2, [pc, #16]	(1c <NVIC_GetSystemHandlerActiveBitStatus+0x1c>)
   a:	6a50      	ldr	r0, [r2, #36]
   c:	ea03 0000 	and.w	r0, r3, r0
D:\STM32\Program\1.11_Odchudzanie\um0427\FWLib\library\src/stm32f10x_nvic.c:668
  10:	4298      	cmp	r0, r3
  12:	bf14      	ite	ne
  14:	2000      	movne	r0, #0
  16:	2001      	moveq	r0, #1
  18:	4770      	bx	lr
  1a:	46c0      	nop			(mov r8, r8)
  1c:	e000ed00 	.word	0xe000ed00
Disassembly of section .text.NVIC_GetFaultHandlerSources:

00000000 <NVIC_GetFaultHandlerSources>:
NVIC_GetFaultHandlerSources():
D:\STM32\Program\1.11_Odchudzanie\um0427\FWLib\library\src/stm32f10x_nvic.c:692
   0:	f3c0 4381 	ubfx	r3, r0, #18, #2
D:\STM32\Program\1.11_Odchudzanie\um0427\FWLib\library\src/stm32f10x_nvic.c:695
   4:	b913      	cbnz	r3, c <NVIC_GetFaultHandlerSources+0xc>
D:\STM32\Program\1.11_Odchudzanie\um0427\FWLib\library\src/stm32f10x_nvic.c:697
   6:	4b0b      	ldr	r3, [pc, #44]	(34 <NVIC_GetFaultHandlerSources+0x34>)
   8:	6ad8      	ldr	r0, [r3, #44]
   a:	e011      	b.n	30 <NVIC_GetFaultHandlerSources+0x30>
D:\STM32\Program\1.11_Odchudzanie\um0427\FWLib\library\src/stm32f10x_nvic.c:699
   c:	2b01      	cmp	r3, #1
   e:	d10d      	bne.n	2c <NVIC_GetFaultHandlerSources+0x2c>
D:\STM32\Program\1.11_Odchudzanie\um0427\FWLib\library\src/stm32f10x_nvic.c:701
  10:	4b08      	ldr	r3, [pc, #32]	(34 <NVIC_GetFaultHandlerSources+0x34>)
D:\STM32\Program\1.11_Odchudzanie\um0427\FWLib\library\src/stm32f10x_nvic.c:693
  12:	f3c0 5101 	ubfx	r1, r0, #20, #2
D:\STM32\Program\1.11_Odchudzanie\um0427\FWLib\library\src/stm32f10x_nvic.c:701
  16:	6a9a      	ldr	r2, [r3, #40]
  18:	00cb      	lsls	r3, r1, #3
  1a:	fa32 f003 	lsrs.w	r0, r2, r3
D:\STM32\Program\1.11_Odchudzanie\um0427\FWLib\library\src/stm32f10x_nvic.c:702
  1e:	2902      	cmp	r1, #2
D:\STM32\Program\1.11_Odchudzanie\um0427\FWLib\library\src/stm32f10x_nvic.c:704
  20:	bf14      	ite	ne
  22:	f000 000f 	andne.w	r0, r0, #15	; 0xf
D:\STM32\Program\1.11_Odchudzanie\um0427\FWLib\library\src/stm32f10x_nvic.c:708
  26:	f000 00ff 	andeq.w	r0, r0, #255	; 0xff
  2a:	e001      	b.n	30 <NVIC_GetFaultHandlerSources+0x30>
D:\STM32\Program\1.11_Odchudzanie\um0427\FWLib\library\src/stm32f10x_nvic.c:713
  2c:	4b01      	ldr	r3, [pc, #4]	(34 <NVIC_GetFaultHandlerSources+0x34>)
  2e:	6b18      	ldr	r0, [r3, #48]
D:\STM32\Program\1.11_Odchudzanie\um0427\FWLib\library\src/stm32f10x_nvic.c:716
  30:	4770      	bx	lr
  32:	46c0      	nop			(mov r8, r8)
  34:	e000ed00 	.word	0xe000ed00
Disassembly of section .text.NVIC_GetFaultAddress:

00000000 <NVIC_GetFaultAddress>:
NVIC_GetFaultAddress():
D:\STM32\Program\1.11_Odchudzanie\um0427\FWLib\library\src/stm32f10x_nvic.c:740
   0:	f410 0f80 	tst.w	r0, #4194304	; 0x400000
D:\STM32\Program\1.11_Odchudzanie\um0427\FWLib\library\src/stm32f10x_nvic.c:742
   4:	bf0c      	ite	eq
   6:	4b03      	ldreq	r3, [pc, #12]	(14 <NVIC_GetFaultAddress+0x14>)
D:\STM32\Program\1.11_Odchudzanie\um0427\FWLib\library\src/stm32f10x_nvic.c:746
   8:	4b02      	ldrne	r3, [pc, #8]	(14 <NVIC_GetFaultAddress+0x14>)
D:\STM32\Program\1.11_Odchudzanie\um0427\FWLib\library\src/stm32f10x_nvic.c:742
   a:	bf0c      	ite	eq
   c:	6b58      	ldreq	r0, [r3, #52]
D:\STM32\Program\1.11_Odchudzanie\um0427\FWLib\library\src/stm32f10x_nvic.c:746
   e:	6b98      	ldrne	r0, [r3, #56]
D:\STM32\Program\1.11_Odchudzanie\um0427\FWLib\library\src/stm32f10x_nvic.c:749
  10:	4770      	bx	lr
  12:	46c0      	nop			(mov r8, r8)
  14:	e000ed00 	.word	0xe000ed00
Disassembly of section .text.NVIC_GetBASEPRI:

00000000 <NVIC_GetBASEPRI>:
NVIC_GetBASEPRI():
D:\STM32\Program\1.11_Odchudzanie\um0427\FWLib\library\src/stm32f10x_nvic.c:250
   0:	b510      	push	{r4, lr}
D:\STM32\Program\1.11_Odchudzanie\um0427\FWLib\library\src/stm32f10x_nvic.c:251
   2:	f7ff fffe 	bl	0 <__GetBASEPRI>
D:\STM32\Program\1.11_Odchudzanie\um0427\FWLib\library\src/stm32f10x_nvic.c:252
   6:	bd10      	pop	{r4, pc}
Disassembly of section .text.NVIC_BASEPRICONFIG:

00000000 <NVIC_BASEPRICONFIG>:
NVIC_BASEPRICONFIG():
D:\STM32\Program\1.11_Odchudzanie\um0427\FWLib\library\src/stm32f10x_nvic.c:235
   0:	b510      	push	{r4, lr}
D:\STM32\Program\1.11_Odchudzanie\um0427\FWLib\library\src/stm32f10x_nvic.c:239
   2:	0100      	lsls	r0, r0, #4
   4:	f7ff fffe 	bl	0 <__BASEPRICONFIG>
D:\STM32\Program\1.11_Odchudzanie\um0427\FWLib\library\src/stm32f10x_nvic.c:240
   8:	bd10      	pop	{r4, pc}
   a:	46c0      	nop			(mov r8, r8)
Disassembly of section .text.NVIC_RESETFAULTMASK:

00000000 <NVIC_RESETFAULTMASK>:
NVIC_RESETFAULTMASK():
D:\STM32\Program\1.11_Odchudzanie\um0427\FWLib\library\src/stm32f10x_nvic.c:221
   0:	b510      	push	{r4, lr}
D:\STM32\Program\1.11_Odchudzanie\um0427\FWLib\library\src/stm32f10x_nvic.c:222
   2:	f7ff fffe 	bl	0 <__RESETFAULTMASK>
D:\STM32\Program\1.11_Odchudzanie\um0427\FWLib\library\src/stm32f10x_nvic.c:223
   6:	bd10      	pop	{r4, pc}
Disassembly of section .text.NVIC_SETFAULTMASK:

00000000 <NVIC_SETFAULTMASK>:
NVIC_SETFAULTMASK():
D:\STM32\Program\1.11_Odchudzanie\um0427\FWLib\library\src/stm32f10x_nvic.c:209
   0:	b510      	push	{r4, lr}
D:\STM32\Program\1.11_Odchudzanie\um0427\FWLib\library\src/stm32f10x_nvic.c:210
   2:	f7ff fffe 	bl	0 <__SETFAULTMASK>
D:\STM32\Program\1.11_Odchudzanie\um0427\FWLib\library\src/stm32f10x_nvic.c:211
   6:	bd10      	pop	{r4, pc}
Disassembly of section .text.NVIC_RESETPRIMASK:

00000000 <NVIC_RESETPRIMASK>:
NVIC_RESETPRIMASK():
D:\STM32\Program\1.11_Odchudzanie\um0427\FWLib\library\src/stm32f10x_nvic.c:197
   0:	b510      	push	{r4, lr}
D:\STM32\Program\1.11_Odchudzanie\um0427\FWLib\library\src/stm32f10x_nvic.c:198
   2:	f7ff fffe 	bl	0 <__RESETPRIMASK>
D:\STM32\Program\1.11_Odchudzanie\um0427\FWLib\library\src/stm32f10x_nvic.c:199
   6:	bd10      	pop	{r4, pc}
Disassembly of section .text.NVIC_SETPRIMASK:

00000000 <NVIC_SETPRIMASK>:
NVIC_SETPRIMASK():
D:\STM32\Program\1.11_Odchudzanie\um0427\FWLib\library\src/stm32f10x_nvic.c:185
   0:	b510      	push	{r4, lr}
D:\STM32\Program\1.11_Odchudzanie\um0427\FWLib\library\src/stm32f10x_nvic.c:186
   2:	f7ff fffe 	bl	0 <__SETPRIMASK>
D:\STM32\Program\1.11_Odchudzanie\um0427\FWLib\library\src/stm32f10x_nvic.c:187
   6:	bd10      	pop	{r4, pc}
